:03000000023D5A64
:0C3D5A0078FFE4F6D8FD75816F023DA1F2
:100E4E0020000A3C2E2E2E3E004950436F6E6E65DA
:100E5E0063745245510A004950436F6E6E65637458
:100E6E00000A49504E6F41434B210A003E432C5617
:100E7E002C52432CC0E4E0EFF2E5F020D1E8EDEA8D
:100E8E00EEEC49500A003E432C4D41432C253032A6
:100E9E0062583A25303262583A25303262583A2535
:100EAE00303262583A25303262583A253032625822
:100EBE002C4D414320E0E4F0E5F10A003E432C5670
:100ECE0045522C20332E3220EEF22025732025732E
:100EDE002CC2E5F0F1E8FF20495020ECEEE4F3EBF4
:100EEE00FF0A004170722031382032303038003124
:100EFE00303A35373A3435003E432C4C442C505260
:100F0E004F473A2020202020202020202020202063
:100F1E0020202020202020202020202020202020C3
:100F2E0020202020202020202020202020202020B3
:100F3E0020202020202020202020202020202020A3
:100F4E0020202020202020202CC4E0F2E020EFF0F2
:100F5E00EEF8E8E2EAE828F4E0E9EB290A003E2A96
:100F6E002C312CCEF1EDEEE2EDFBE520EFE0F0E0E2
:100F7E00ECE5F2F0FB20F1E5F2E5E2EEE3EE20E83F
:100F8E00EDF2E5F0F4E5E9F1E00A003E412C4130E6
:100F9E00312C2562752E2562752E2562752E2562E1
:100FAE00752C495020E0E4F0E5F120E0E4E0EFF2AA
:100FBE00E5F0E00A003E412C4130322C2562752EC0
:100FCE002562752E2562752E2562752C495020E0FE
:100FDE00E4F0E5F120EEF1ED2E20F1E5F0E2E5F0A2
:100FEE00E00A003E412C4130332C2562752E2562DD
:100FFE00752E2562752E2562752C495020E0E4F081
:10100E00E5F120F0E5E72E20F1E5F0E2E5F0E00A6B
:10101E00003E412C4130342C2562752E2562752EF2
:10102E002562752E2562752CCCE0F1EAE020F1E503
:10103E00F2E80A003E412C4130352C2562752E25F2
:10104E0062752E2562752E2562752CD8EBFEE70A89
:10105E00003E2A2C312CC4EEEF2E20EFE0F0E0EC17
:10106E00E5F2F0FB20F1E5F2E5E2EEE3EE20E8ED4D
:10107E00F2E5F0F4E5E9F1E00A003E422C5330319E
:10108E002C2562752CC6E4E0F2FC20E7E0EFF0EED2
:10109E00F1E020F1EEE5E4E8EDE5EDE8FF20EEF21B
:1010AE0020F1E5F0E2E5F0E00A003E422C5330324A
:1010BE002C2562752CCEE1ECE5ED20F120F1E5F06A
:1010CE00E2E5F0EEEC20E1E5E720EAE2E8F2E0ED21
:1010DE00F6E8E90A003E422C5330332C2562752C7B
:1010EE00CFE5F0E5E7E0EFF3F1EA20EFF0E820EFEF
:1010FE00EEF2E5F0E520F1E2FFE7E820F120F1E580
:10110E00F0E2E5F0EEEC0A003E422C5330352C2591
:10111E0062752CCAE0EDE0EB20F8E8F0EEEAEEE2C4
:10112E00E5F8E0F2E5EBFCEDEEE3EE20EEE1ECE5CA
:10113E00EDE00A003E532C5330362C2530326258E7
:10114E0025303262582530326258253032625825A9
:10115E003032625825303262582C4D414320E0E443
:10116E00F0E5F120F8E8F0EEEAEEE2E5F8E0F2E57F
:10117E00EBFCEDEEE3EE20EEE1ECE5EDE00A003EF9
:10118E00454E440A000A44756D70582020202020D8
:10119E003030203031203032203033203034203087
:1011AE00352030362030372030382030392030414D
:1011BE00203042203043203044203045203046003D
:1011CE000A3A003A20000A000A44756D7044202045
:1011DE00202020303020303120303220303320306B
:1011EE00342030352030362030372030382030391A
:1011FE0020304120304220304320304420304520E2
:10120E00304600457272206B657900526420656528
:10121E0070726F6D0A005264204D454D0A00526483
:10122E0020436F64650A00577269746520436F64CA
:10123E00650A0044656275674950204F4E0A0044A6
:10124E00656275674950204F46460A0044656275CF
:10125E006755736572204F6E0A0044656275675557
:10126E00736572204F46460A0044656275674D737A
:10127E0067204F6E0A0044656275674D7367204F95
:10128E0046460A00436F6E666967206C6F636B217A
:10129E000A00577220656570726F6D0A00205361E7
:1012AE00766520656570726F6D210A004572722039
:1012BE004D414321004C6F61643E3E002A003C418B
:1012CE0030313D003C4130323D003C4130333D0039
:1012DE003C4130343D003C4130353D003C21003C2A
:1012EE005330313D003C5330323D003C5330333DA2
:0D12FE00003C5330353D003C5330363D0080
:06483300010B0001090069
:1047C900C28E438910758BFF758DB7D2ABD28E22FD
:03001B00023C3A6A
:103C3A00C0E0C083C082C0D0C28E758BFF758DB7BD
:103C4A0020060675A61E75A6E10509D202E50B60D7
:103C5A0002050BE50AD394014002150A050EE50E8A
:103C6A00540F7048D20EE50E543F7012D200907A6B
:103C7A00EFE0600A04F0E0D394B44002D206907AEE
:103C8A00EAE0600204F0907568E0600214F0907A4D
:103C9A00F0E0D394014003E014F0300502050CE58E
:103CAA000DD394644004D2068002050DE508D3942E
:103CBA000140021508D28ED0D0D082D083D0E03213
:10088100C2AFC20B7D027C007F0712477B8F26E53A
:1008910026646060097D017F601246CED20BE4FDC3
:1008A100FC7F0B12477B8F26E52630E6097D04E4A9
:1008B100FF1246F2D20B7D017C007F0712477B8F2E
:1008C10026E5267008FD7FFF1246CED20B300B03C2
:1008D100126000C288C2A8C2AA758900123B0590A5
:1008E10077AD7403F0A374CCF0E49077ACF01238D8
:1008F100E112235FC2061243A2D20BC20DC20C90B9
:1009010079DA7408F09077187424F0E4A3F0907702
:10091100A2E090771AF09077A3E090771BF09077A0
:10092100A4E090771CF09077A5E090771DF0907788
:10093100A6E090771EF09077A7E090771FF0750AF8
:1009410001E49079DBF0C207C208C209C20A12466B
:10095100A7200B19AF267E007D0312356CE4FF1230
:1009610039AB7E0E7F4EE4FBFDFC123173907AEFC2
:10097100E060037401F0E4907568F0F50C9079D9AA
:10098100F0F50D1247C975A70775A61E75A6E1D228
:10099100AFE4F50D907568E07003121E1B907AF0BC
:1009A100E0B401119080007410F0E4907AF0F0D27C
:1009B1000BC20CC20D908008E0F52630E405D20789
:1009C1007410F0E52630E508D2099080087420F013
:1009D100E52630E608D2089080087440F0E50CC3A3
:1009E10094034019908002E4F0908001F09080001F
:1009F100F0E50C94064006E4F50C1243A29080A0A9
:100A0100E070031241939080B8E0700312420D90A0
:100A110080D0E07003124287908000E070133007AD
:100A210010123380907795EFF0D3940040031200B9
:100A310026908002E07006908000E06005D20502F9
:100A41000992C205E4F50C907568E0600302099211
:100A5100200B129079DCE0600C7E0E7F5012348402
:100A6100E49079DCF0300912122DB0907795EFF017
:100A7100D394004005E0FF1247E8200803020BF67B
:100A8100122AB7907795EFF070030209929077D907
:100A9100E054BF247F7003020B5F147003020B3715
:100AA10024026003020B98200B077E0E7F5712343D
:100AB10084200F03020BF69077B1E0FF7006907768
:100AC100B5E06061907AE6E0FEB50722A3E0FF9011
:100AD10077B2E0B50718907AE8E0FF9077B3E0B518
:100AE100070C907AE9E0FF9077B4E06F6037907778
:100AF100B5E06E6003020BF6907AE7E0FF9077B6FF
:100B0100E06F6003020BF6907AE8E0FF9077B7E0C0
:100B11006F6003020BF6907AE9E0FF9077B8E06F1F
:100B21006003020BF6C2039079DB7401F01200211D
:100B3100750A01020BF6907AEFE060037401F09000
:100B41007ADEE0FF9077DBE06F6003020BF6907ACC
:100B5100DEE004F0E4F50A9079D9F0020BF63003F7
:100B610003020BF69077A8E070030209929077B91F
:100B7100740AF0124848D203E4F50A9079D9F0904A
:100B81007AEA04F0E4907ADDF0A3F0200B677E0EA0
:100B91007F65123484805E907AEFE060037401F027
:100BA1003003529077D9E020E74B9077DBE0FF905C
:100BB1007ADDE0FE6F600D907AE5E07007EE146F6C
:100BC10070338013907ADDE004F0907795E0FFD3E5
:100BD100940440031244CB9074647482F0A37401B2
:100BE100F09077DBE0907466F07E747F647D031291
:100BF1003EF9020992200303020D0EE50A70681204
:100C01004575EF60237E787FD99078DAE02404FD82
:100C1100123EF9907AE5E070099077B9E0F50A02A1
:100C21000992E4F50A020992907AEAE0D3943C40F1
:100C310036907AE5E07030907AEA04F0124829E4BF
:100C41009078D9F0A37412F0907ADEE09078DBF01E
:100C5100A374FDF090756963A2019078DD63A20130
:100C61007F1212263D809E12481E8F26E526B40172
:100C7100159074647483F0E4A3F07E747F647D0244
:100C8100123EF9020992E526D39401401C90746446
:100C91007483F0A37401F0E52624FEA3F07E747F33
:100CA100647D03123EF9020992E50A6401600302C0
:100CB10009929079D9E004F0200B077E0E7F6F1224
:100CC10034849077B9E0C394C85004E02432F090A2
:100CD10079D9E0C39405400DC203E49079DBF012A9
:100CE10000210209927C7A7DE69077ADE0FAA3E0DB
:100CF100FB7F0212410F7E787FD99078DAE02404DD
:100D0100FD123EF99077B9E0F50A020992E50A640D
:100D11000160030209929079DBE014604624FE60D1
:100D210042147003020E0124046003020992E4F5E7
:100D31000C200F139079DB7404F09079D9E0540101
:100D4100F0750A010209929080027410F0E4907922
:100D5100DBF09079D904F0750AFA907AE674FFF025
:100D6100020992907AE6E07003020DEB9078D97453
:100D710080F09078DB7401F0E4A3F0A304F0A37495
:100D810030F0A3747BF0E4F52674E02526F582E4C7
:100D91003478F583747DF074E12526F582E43478A6
:100DA100F583E4F0E52624079078DAF07C7A7DE695
:100DB1009077ADE0FAA3E0FB7F0212410F7E787FCE
:100DC100D9E5262409FD123EF9907AE5E0601B126F
:100DD1004848D203E4F50A9079D9F0907AEA04F010
:100DE100E4907ADDF0A3F0020992300F07E49079E4
:100DF100DBF080069079DB7404F0750AFA0209923F
:100E01009080027410F0750A059079D9E06401FFB1
:100E1100F09079DB7401F0EF70199077B5E0601311
:100E2100FCA3E0FDA3E0FEA3E0FF907AE612221509
:100E31000209929077B1E0FCA3E0FDA3E0FEA3E0FC
:0C0E4100FF907AE612221502099280FE52
:010E4D002282
:100026009077DAE0B444047F0180027F009077D9AC
:10003600E0B447047E0180027E00EE5F604A90775E
:10004600A2E09077DBF09077A3E09077DCF09077F2
:10005600A4E09077DDF09077A5E09077DEF09077DA
:10006600A6E09077DFF09077A7E09077E0F09077C2
:10007600DA7452F090771263A2019080A863A2010D
:100086007F0612263D020877907795E0C3940850C4
:10009600030208809077A2E0FF9077DBE06F6003B1
:1000A6000208809077A3E0FF9077DCE06F600302A0
:1000B60008809077A4E0FF9077DDE06F6003020888
:1000C600809077A5E0FF9077DEE06F6003020880FE
:1000D6009077A6E0FF9077DFE06F600302088090DC
:1000E60077A7E0FF9077E0E06F60030208809077E3
:1000F600DAE0B44415907712E0B4FF0E63A20190E3
:1001060080A863A2017F0612263D907AEFE0600385
:100116007401F0907AF07464F09077DA7452F0908B
:1001260077D9E0646D60030202857BFF7A0E797AE7
:100136001218277BFF7A0E79949077A2E0F52FA309
:10014600E0F530A3E0F531A3E0F532A3E0F533A303
:10015600E0F534121827752FFF75300E7531F175DD
:1001660032FF75330E7534FD7BFF7A0E79CA12188D
:10017600277BFF7A0F79061218277BFF7A0F796C97
:100186001218277BFF7A0F79999077A8E0F52FA3AD
:10019600E0F530A3E0F531A3E0F5321218277BFF36
:1001A6007A0F79C39077B1E0F52FA3E0F530A3E09D
:1001B600F531A3E0F5321218277BFF7A0F79F1901B
:1001C60077B5E0F52FA3E0F530A3E0F531A3E0F530
:1001D600321218277BFF7A10791F90779EE0F52F51
:1001E600A3E0F530A3E0F531A3E0F5321218277B42
:1001F600FF7A10794290779AE0F52FA3E0F530A3C5
:10020600E0F531A3E0F5321218277BFF7A10795F0B
:100216001218277BFF7A107988A20FE433F52F1284
:1002260018277BFF7A1079B8907AE5E0F52F121837
:10023600277BFF7A1079E3907AEFE0F52F121827E3
:100246007BFF7A117916A201E433F52F1218277B6A
:10025600FF7A117942907ADFE0F52FA3E0F530A31B
:10026600E0F531A3E0F532A3E0F533A3E0F534126F
:100276001827123A5B7BFF7A11798D121827229084
:1002860077D9E0644C70737E117F93FBFDFC1231CD
:10029600739077E1E0F527A3E0F528E4F52AE52752
:1002A6009077E3F0A3E528F07E117FCE7C777DE39F
:1002B6007B02123173E4F529852882852783E0FFC6
:1002C60074E32529F582E43477F583EFF00528E514
:1002D60028700205270529E529B410DC7E117FD197
:1002E6007C777DE37B10123173052AE52AC39410CF
:1002F60040AC7E117FD4123484229077D9E0646CAE
:100306007060F52B7E117FD6FBFDFC123173E4F590
:100316002AE49077E3F0A3E52BF07E117FCE7C777D
:100326007DE37B02123173E4F529A82BE6FF74E323
:100336002529F582E43477F583EFF0052B0529E5C9
:1003460029B410E67E117FD17C777DE37B101231D4
:1003560073052AE52AC3940840B77E117FD4123468
:1003660084229077D9E0644B7061F52974CB2529F6
:10037600F582E43477F583E0603274CB2529F58283
:10038600E43477F583E0F4602374CB2529F582E421
:100396003477F583E0FF74E12529F582E43477F5B7
:1003A60083E0B507100529E529B408C0907568747F
:1003B60032F00208779077D97421F0300B030208E7
:1003C600777E127F111234840208779077D9E0B4D1
:1003D600521A200B077E127F191234849077D97433
:1003E60072F07E777FD97D08123E72229077D9E02F
:1003F60064497045200B077E127F2412348490775F
:10040600E1E0F527A3E0F528E4F52985288285278C
:1004160083E0FF74E32529F582E43477F583EFF072
:100426000528E528700205270529E529B480DC7E24
:10043600777FD97D8A123E72229077D9E064437025
:1004460046200B077E127F2C1234849077E1E0F56C
:1004560027A3E0F528E4F529852882852783E493F8
:10046600FF74E32529F582E43477F583EFF0052858
:10047600E528700205270529E529B480DB7E777F0C
:10048600D97D8A123E72229077D9E0645A70532041
:100496000B077E127F351234849077E1E0F527A3AF
:1004A600E0F5287C777DE37B80AF28AE27124541B7
:1004B600E4F529852882852783E493FF74E32529BB
:1004C600F582E43477F583EFF00528E52870020518
:1004D600270529E529B480DB7E777FD97D8A123E00
:1004E60072229077D9E0644460030205799077E13F
:1004F600E0FF64447003020877EFB4310CC20B7E50
:10050600127F411234840208779077E1E0B4300C10
:10051600D20B7E127F4D1234840208779077E1E089
:10052600B4320CD20C7E127F5A12348402087790B1
:1005360077E1E0B4330CC20C7E127F681234840279
:1005460008779077E1E0B4340CD20D7E127F7712F3
:1005560034840208779077E1E0B4350CC20D7E1240
:100566007F841234840208779077E1E0FF12001E40
:10057600020877907568E07013200B077E127F9251
:100586001234849077D97421F002087790756874D4
:1005960032F09077D9E0FFB45104C2AF80FEEF6429
:1005A600577045200B077E127FA01234849077E2A5
:1005B600E0907795F0E4F529907795E0FFE529C37B
:1005C6009F400302087774E32529F582E43477F522
:1005D60083E0FF9077E1E025292411F582E4347663
:1005E600F583EFF0052980D09077D9E06453600356
:1005F60002069B200B077E127FAB1234849077A2F3
:10060600E0FF90761AE06F703C9077A3E0FF90765B
:100616001BE06F70309077A4E0FF90761CE0B50782
:10062600249077A5E0FF90761DE0B507189077A691
:10063600E0FF90761EE0B5070C9077A7E0FF907676
:100646001FE06F60169077D97421F0300B03020813
:10065600777E127FBA123484020877E4F529E4F52E
:100666000D74112529F582E43476F583E0FDAF2972
:100676001246020529E529C394FE40E2C2AFE49082
:100686007FF0F0A3F0907FFD74AAF0A374FFF0A3AF
:100696007455F080FE9077D9E0644F704C9077E106
:1006A600E0F527A3E0F528E5284527700A200B0783
:1006B6007E127FC3123484200B077E127FCA123447
:1006C60084E4F52974E32529F582E43477F583E09B
:1006D600852882852783F00528E5287002052705E9
:1006E60029E529B480DE0208779077D9E0FFB44582
:1006F600219077E1E0FDA3E0907FF0CDF0A3EDF04F
:10070600C2AF907FFD74AAF0A374FFF0A37455F0F6
:1007160080FEEF646560030208809077E1E0FFA346
:10072600E0907FF0CFF0A3EFF0E4F527F528D39023
:100736007FF1E09528907FF0E095274021E4F50DC4
:100746002528FFE5273478FE7B80AD28AC271245A7
:100756004174802528F528E43527F52780D07E12B8
:100766007FCC123F80EF4E60201200039077A8EFF7
:10077600F01200039077A9EFF01200039077AAEF2A
:10078600F01200039077ABEFF07E127FD2123F801B
:10079600EF4E60201200039077B1EFF01200039045
:1007A60077B2EFF01200039077B3EFF012000390E8
:1007B60077B4EFF07E127FD8123F80EF4E602012A2
:1007C60000039077B5EFF01200039077B6EFF012C2
:1007D60000039077B7EFF01200039077B8EFF07E42
:1007E600127FDE123F80EF4E602012000390779E4C
:1007F600EFF012000390779FEFF01200039077A0BE
:10080600EFF01200039077A1EFF07E127FE4123F23
:1008160080EF4E602012000390779AEFF0120003EB
:1008260090779BEFF012000390779CEFF012000395
:1008360090779DEFF0E4F529E4F50DE52904FF74C2
:100846009A2529F582E43477F583E0FD1246020500
:1008560029E529C3944340E0C2AFE4907FF0F0A3BA
:10086600F0907FFD74AAF0A374FFF0A37455F08096
:0A087600FE7E777FD97D08123E72E6
:010880002255
:10450900AE07EEC39430400BEED394395005EE2438
:10451900D0FF22EEC39461400BEED394665005EEB2
:1045290024A9FF22EEC39441400BEED394465005D3
:08453900EE24C9FF22AF0622A7
:10479800907711E004F07006907710E004F09077BD
:0A47A80010E0FEA3E0FF1244892296
:10000300124798124509EFC454F0FEC006124798F0
:08001300124509D0E02FFF2285
:1042EA00E4907C31F0124798907C32EFF0C394301E
:1042FA004018E0FFD394395011907C31E02469F5DD
:10430A0082E43475F583EFF08011907C31E0246902
:10431A00F582E43475F583E4F0800C907C31E00496
:10432A00F0E0D3940840BE752E00752F007530005A
:0C433A00E4F5317B017A757969122913D2
:014346002254
:043F80008E2C8F2DC7
:103F8400907710E4F0A374FFF0124798EF606EF49A
:103F9400606B852D82852C83E493B507EC752E0127
:103FA400E52D252EF582E4352CF583E493602590E8
:103FB4007711E0252EFF907710E03400FE1244893B
:103FC400E52D252EF582E4352CF583E493B507041D
:103FD400052E80CCE52D252EF582E4352CF583E4E1
:103FE4009370A6E52E24FFFFE434FFFE907711E0E2
:103FF4002FF0907710E03EF07E007F0122E4FEFF78
:014004002299
:1038E1007E127FEA123F80EF4E70037F01227E122B
:1038F1007FED123F80EF4E600C124798EF24D024E9
:10390100FF920F8002D20F7E127FF3123F80EF4EA3
:10391100600C124798EF24D0907AE5F08005E4908E
:103921007AE5F07E127FF9123F80EF4E600C12476C
:1039310098EF24D0907AEFF08005E4907AEFF07E52
:10394100127FFF123F80EF4E600C124798EF24D098
:1039510024FF92018002C2019077A263A201907AB2
:10396100DF63A2017F0612263D30013B7E137F05F6
:10397100123F80EF4E6030120003907ADFEFF012B9
:103981000003907AE0EFF0120003907AE1EFF01279
:103991000003907AE2EFF0120003907AE3EFF01265
:0A39A1000003907AE4EFF07F0022AB
:1043FB009079DAE0C3947C503D9079DAE0FE04F0DA
:10440B0074182EF582E43477F583EFF0BF0A27900A
:10441B0079DAE0FF04F074182FF582E43477F58332
:10442B00E4F09079DAE0FF1240059079DA7408F045
:07443B00907719E004F02264
:1043A2009080007480F090779A63A201F583F58281
:1043B20063A2017F0812263D9077A263A20190803A
:1043C2008863A2017F0A12263D908092E4F0A374D2
:1043D20032F0A37401F09077ACE0FF9080B1F090DE
:1043E20080E1EFF09080957455F0A3F09080007416
:0943F20001F090800974F0F02242
:10419300908009E04410F09080A0E0706C9080A1C2
:1041A3007482F09080A874FFF0A3F0A3F0A3F07FD3
:1041B300039080AEEFF07FCBA3EFF07F039080AC52
:1041C300EFF0A374CBF09080007402F0907C231284
:1041D300222100000000907C23E0908040F0907C3E
:1041E30024E0908041F0907C25E0908042F0907C28
:1041F30026E0908043F0A3E4F0A3F0A3F0A3F090B3
:094203008018F0A3F0A3F0A3F071
:01420C00228F
:10428700908009E04440F09080D17482F09077AD3F
:10429700E0FF9080DEF09077AEE0FF9080DFF09057
:1042A70080027402F0907C27122221000000009007
:1042B7007C27E0908058F0907C28E0908059F0901F
:1042C7007C29E090805AF0907C2AE090805BF0A3F4
:1042D700E4F0A3F0A3F0A3F0908030F0A3F0A3F0F4
:0242E700A3F042
:0142E90022B2
:10420D00908009E04420F09080B8E0706C9080B907
:10421D007482F07F039080C6EFF07FCDA3EFF07F27
:10422D00039080C4EFF0A374CDF09080C074FFF0C4
:10423D00A3F0A3F0A3F09080017402F0907C2B12F8
:10424D00222100000000907C2BE090804CF0907CAF
:10425D002CE090804DF0907C2DE090804EF0907C85
:10426D002EE090804FF0A3E4F0A3F0A3F0A3F09024
:09427D008024F0A3F0A3F0A3F0EB
:014286002215
:10410F008C278D28A907EAFDE975F018A424ACFFC8
:10411F00E5F034808F82F583EDF0EBFDE975F01853
:10412F00A4FFAEF024ACFBEE34808B82F583A3EDBD
:10413F00F08528828C83E0FDEF24A8FFEE3480FE0B
:10414F008F82F583EDF08528828C83A3E08F828E9A
:10415F0083A3F0852882852783A3A3E0FDE975F06B
:10416F0018A424A8FFE5F03480FE8F82F583A3A363
:10417F00EDF08528828C83A3A3A3E08F828E83A387
:04418F00A3A3F022D4
:063E72008D2CAB07AA062F
:103E7800908000E030E5079079DC7401F022907CB6
:103E880023E0FCA3E0FDA3E0FEA3E0F5308E2F8D38
:103E98002E8C2DAE02AF038E838F8263A201E52F95
:103EA800540744C0F58385308263A201AF2C1226E3
:103EB800AFE4FCFDFEE530252CF530EE352FF52F6F
:103EC800ED352EF52EEC352DF52D908040E52DF0B5
:103ED800A3E52EF0A3E52FF0A3E530F09080007461
:103EE80020F0AF30AE2FAD2EAC2D907C23122215D2
:013EF80022A7
:063EF9008D27AB07AA06AD
:103EFF00908002E030E5079079DC7403F022907C2B
:103F0F0027E0FCA3E0FDA3E0FEA3E0F52B8E2A8DB6
:103F1F00298C28AE02AF038E838F8263A201E52A1C
:103F2F00540744D0F583852B8263A201AF27122655
:103F3F00AFE4FCFDFEE52B2527F52BEE352AF52A00
:103F4F00ED3529F529EC3528F528908058E528F02E
:103F5F00A3E529F0A3E52AF0A3E52BF090800274E6
:103F6F0020F0AF2BAE2AAD29AC28907C271222155A
:013F7F00221F
:0239AB008F2863
:1039AD00908001E030E5099079DC7402F07F00220F
:1039BD00907C2BE0FCA3E0FDA3E0FEA3E0F52C8EB4
:1039CD002B8D2A8C29907ADF63A201E52B540744B5
:1039DD00C8F583852C8263A2017F061226C5E52CCE
:1039ED002406F52CE4352BF52BE4352AF52AE435A0
:1039FD0029F5299079DD63A201E52B540744C8F51B
:103A0D0083852C8263A201AF281226C5E4FCFDFE3E
:103A1D00E52C2528F52CEE352BF52BED352AF52A41
:103A2D00EC3529F52990804CE529F0A3E52AF0A382
:103A3D00E52BF0A3E52CF09080017420F0AF2CAEB7
:0D3A4D002BAD2AAC29907C2B122215AF283E
:013A5A002249
:103380009081E0E0F5270527052705270527052774
:1033900005270527052705270527908010E0F52A32
:1033A000A3E0F52BA3E0F52CA3E0F52D9081E1E05F
:1033B000F5270527052705270527052705270527BD
:1033C000052705270527908014E0F52EA3E0F52FAB
:1033D000A3E0F530A3E0F531E530B52C08E531B5D3
:1033E0002D037F0022E4F527E530540744E0F58300
:1033F00085318263A2019077D963A2017F081226EA
:10340000F59077DB63A20190771263A2017F061229
:10341000263D9077D9E0F528A3E0F529E4F527903B
:1034200077D9E0702AA3E024F8F527E53054074463
:10343000E0F58385318274082582F582E43583F5D1
:103440008363A2019077D963A201AF271226F5AE5C
:1034500028E4FCFDE5312529F531E5303EF530ED78
:10346000352FF52FEC352EF52E908014E52EF0A398
:10347000E52FF0A3E530F0A3E531F0908000744033
:03348000F0AF2783
:013483002226
:102AB7009081E6E0F5270527052705270527052740
:102AC70005270527052705270527908028E0F52AEC
:102AD700A3E0F52BA3E0F52CA3E0F52D9081E7E02B
:102AE700F52705270527052705270527052705278F
:102AF70005270527052790802CE0F52EA3E0F52F65
:102B0700A3E0F530A3E0F531E4F527E530B52C0A6D
:102B1700E531B52D05C208022C23E530540744F0F2
:102B2700F58385318263A2019077D963A2017F087B
:102B37001226F59077D9E0F528A3E0F529E5294590
:102B47002870099080027410F07F0022907AE6E0E6
:102B5700FFF460309077DBE06F6003022BEA907A36
:102B6700E7E0FF9077DCE06F7079907AE8E0FF901C
:102B770077DDE06F706D907AE9E0FF9077DEE06FC8
:102B87006031805F9077DBE0907AE6F09077DCE069
:102B9700907AE7F09077DDE0907AE8F09077DEE0E2
:102BA700907AE9F09077DFE0FFA3E09077ADCFF080
:102BB700A3EFF09077D9E0702AA3E024F8F527E592
:102BC70030540744F0F58385318274082582F582F5
:102BD700E43583F58363A2019077D963A201AF2718
:102BE7001226F5AE28E4FCFDE5312529F531E5305F
:102BF7003EF530ED352FF52FEC352EF52EAF2DAEFA
:102C07002CAD2BAC2AAB31AA30A92FA82ED3122278
:102C17000440099080027410F07F002290802CE518
:102C27002EF0A3E52FF0A3E530F0A3E531F0908077
:062C3700027440F0AF271B
:012C3D002274
:102DB0009081E3E0F5270527052705270527052747
:102DC0000527052705270527052790801CE0F52AFC
:102DD000A3E0F52BA3E0F52CA3E0F52D9081E4E032
:102DE000F527052705270527052705270527052793
:102DF000052705270527908020E0F52EA3E0F52F75
:102E0000A3E0F530A3E0F531E4F527E530B52C0A71
:102E1000E531B52D05C209022EFBE530540744E823
:102E2000F58385318263A20190746863A2017F0EED
:102E300012270B907468E0F528A3E0F529907470D0
:102E4000E0FFF46045907ADFE0FEEF6E706EA3E085
:102E5000FF907471E06F7064907AE1E0FF9074729B
:102E6000E06F7058907AE2E0FF907473E06F704CFE
:102E7000907AE3E0FF907474E06F7040907AE4E041
:102E8000FF907475E06F60048032D2D9907468E06E
:102E9000702AA3E024F2F527E530540744E8F583CF
:102EA000853182740E2582F582E43583F58363A231
:102EB0000190746863A201AF2712270BAE28E4FCCF
:102EC000FDE5312529F531E5303EF530ED352FF5BD
:102ED0002FEC352EF52EAF2DAE2CAD2BAC2AAB3111
:102EE000AA30A92FA82ED31222045006E52945287E
:102EF00070099080017410F07F0022908020E52EF0
:102F0000F0A3E52FF0A3E530F0A3E531F0908001C8
:052F10007440F0AF2742
:012F15002299
:043484008E2C8F2DCE
:10348800908000E030E5079079DC7401F022907CB0
:1034980023E0FCA3E0FDA3E0FEA3E0F5338E328D2C
:1034A800318C30E533FFE5325407FEE42FF52FEE7B
:1034B80034C0F52E852F82F5837423F0052FE52F70
:1034C8007002052E532EC7F582852E83740AF005E7
:1034D8002FE52F7002052E532EC79077A263A20105
:1034E800852E83852F8263A2017F061226AF74067C
:1034F800252FF52FE4352EF52E852C83852D826317
:10350800A201852E83852F8263A201122693E4FCF3
:10351800FDFE907C23E0F8A3E0F9A3E0FAA3E02FF6
:10352800FFEE3AFEED39FDEC38FCEF2408FFE43EEF
:10353800FEE43DFDE43CFC907C23122215907C23A4
:10354800E0908040F0907C24E0908041F0907C25D1
:10355800E0908042F0907C26E0908043F0908000DC
:033568007420F0DC
:01356B00223D
:0A3173008E2C8F2D8C2E8D2F8B30AB
:10317D00908000E030E5079079DC7401F022907CBE
:10318D0023E0FCA3E0FDA3E0FEA3E0F5368E358D34
:10319D00348C33E536FFE5355407FEE42FF532EE7A
:1031AD0034C0F531853282F5837423F00532E53272
:1031BD00700205315331C7F582853183740AF005EC
:1031CD0032E532700205315331C79077A263A20107
:1031DD0085318385328263A2017F061226AF740684
:1031ED002532F532E43531F531852C83852D826319
:1031FD00A20185318385328263A2011226938F3716
:10320D00EF2532F532E43531F531E5306017852E95
:10321D0083852F8263A20185318385328263A2016A
:10322D00AF301226AFE53724082530F530FFE4FC2A
:10323D00FDFEE5362FF536EE3535F535ED3534F544
:10324D0034EC3533F533908040E533F0A3E534F0BD
:10325D00A3E535F0A3E536F09080007420F0AF368D
:0C326D00AE35AD34AC33907C231222153A
:013279002232
:024005008F40EA
:10400700908000E030E5079079DC7401F022907C25
:1040170023E0FCA3E0FDA3E0FEA3E0F5448E438D7F
:10402700428C41E544FFE5435407FEE42FFFEE349D
:10403700C090771863A201F5838F8263A201AF4016
:104047001226AFE4FCFDFEE5442540F544EE35437A
:10405700F543ED3542F542EC3541F541908040E5B9
:1040670041F0A3E542F0A3E543F0A3E544F09080D7
:10407700007420F0AF44AE43AD42AC41907C2312B4
:02408700221500
:014089002214
:06356C008E2B8F2CAB0535
:10357200908000E030E5079079DC7401F022907CC5
:1035820023E0FCA3E0FDA3E0FEA3E0F5328E318D43
:10359200308C2FE532FFE5315407FEE42FF52EEE95
:1035A20034C0F52D852E82F5837423F0052EE52E89
:1035B2007002052D532DC7F582852D83EBF0052E64
:1035C200E52E7002052D9077A263A201852D8385D9
:1035D2002E8263A2017F061226AF7406252EF52ED7
:1035E200E4352DF52D532DC7E52B852E82852D83B0
:1035F200F0052EE52E7002052D532DC7F582852D7F
:1036020083E52CF0052EE52E7002052D532DC7E51E
:1036120032240AF532E43531F531E43530F530E45F
:10362200352FF52F908040E52FF0A3E530F0A3E58C
:1036320031F0A3E532F09080007420F0AF32AE3169
:0A364200AD30AC2F907C231222154E
:01364C00225B
:103B0500E4F527E5272401FFE433FE124489749A7E
:103B15002527F582E43477F583EFF00527E527C3FC
:103B2500943F40DFE4F527E527247FFFE433FE12C9
:103B3500448974912527F582E43475F583EFF07493
:103B4500912527F582E43475F583E0FF6003B4FF22
:103B55001D74912527F582E43475F5837420F0747E
:103B6500922527F582E43475F583E4F0800905276D
:103B7500E527C3948040B0E4907610F0F527AF2791
:103B85007E0012448974112527F582E43476F58385
:0B3B9500EFF00527E527C394FE40E396
:013BA0002202
:10475B00E4FDFCC3ED9FEC9E5015E4FBFA0BBB0094
:0F476B00010ABA01F8BB90F50DBD00010C80E406
:01477A00221C
:0D47F7004390014390025390FE5390FD2229
:0D4804005390FD5390FE439002439001221B
:0E47D9005390FD439002E5905408FF5390FD6D
:0147E70022AF
:0D4811005390FD4390014390025390FD220F
:07483A00AE071FEE70FA2229
:0245D600AD072F
:1045D800E4FC5390FDEDA804088002C333D8FC30F6
:1045E800E70543900180035390FE7F0512483A4344
:0945F80090020CBC08DC5390FD9C
:014601002296
:10465600E4FF5390FD7E07439002E59030E00D7431
:1046660001A806088002C333D8FC42075390FD1EFA
:08467600C3EE6480948050DF64
:01467E002219
:10460200AB05AA071247F77FA01245D61247D9AFCA
:10461200021245D61247D9AF031245D61247D91214
:0A46220048047F0A7E0012475B2265
:04448900AB07AA06CD
:10448D00C3EB94FFEA9400400DE42BF58274773A68
:10449D00F583E493FF221247F77FA01245D612470A
:1044AD00D9AF031245D61247D91247F77FA112454E
:0D44BD00D61247D912465612481112480473
:0144CA0022CF
:024541008B2CC1
:10454300A2AF921EC2AF85A22D53A2FE8E838F828D
:1045530005A28C838D827409122739E52C53A2FEA0
:1045630043A22012273B53A2DF852DA2A21E92AFA6
:01457300FF48
:014574002224
:10477B00A2AF921EC2AF8C838D82EF12273943A258
:0C478B002012273B53A2DFA21E92AFFFBA
:0147970022FF
:0246CE008F2734
:1046D000A2AF921EC2AFE4F5838D82740612273911
:1046E000E52743A22012273B53A2DFA21E92AF7FF1
:0146F00001C8
:0146F10022A6
:0246F2008F2710
:1046F400A2AF921EC2AFE4F5838D82740A122739E9
:10470400E52743A22012273B53A2DFA21E92AF7FCC
:0147140001A3
:014715002281
:10256200A907E7FFA805EF93C3966008403B74FCF8
:102572002FFF80F00F08EF93C3966008402B74FB87
:102582002FFF80E00F08EF93C3966008401B74FA98
:102592002FFF80D00F08EF93D3966008400B74F999
:1025A2002FFF80C01F1F1F1F1FEF54FEF80303F7EA
:1025B200E893FC08E893FD08E893FE08E893FF22FD
:1025C20009E993C39D6008402974FB29F980F10948
:1025D200E993C39E6008401A74FA29F980E209E976
:1025E20093D39F6008400B74F929F980D319191904
:1025F2001919E9C313C313FF22740093F8ECC398AB
:102602004024701F740193F8EDC39840197014743C
:0E2612000293F8EEC398400E7009740393F81B
:10262000EFC39840037F00227F0122EDF8E6F00817
:10263000A3DFFA22EDF8E0F608A3DFFA22E0A363B5
:10264000A201F0A363A201DFF475A2002263A2013C
:10265000F0A363A20122E0A363A201F0A363A2019D
:10266000E0A363A201F0A363A201E463A201F0A3CB
:1026700063A201DFE175A20022E0A363A2016DFE67
:10268000936CFDEE058393FC158363A201DFEA756D
:10269000A200227F00E493A363A201F00F600CA3C9
:1026A000E583C2E3F58363A20180EA75A20022E01C
:1026B000A363A201F0A3E583C2E3F58363A201DF74
:1026C000EE75A20022E0A363A201F0A3E583C2E4B9
:1026D000D2E3F58363A201DFEC75A20022E0A363DD
:1026E000A201F0A3E58344F8C2E5F58363A201DF0C
:1026F000EC75A20022E583C2E3F583E0A363A201A7
:10270000F0A363A201DFEE75A20022E583C2E4D24A
:0A271000E3F583E0A363A201F0A348
:10271A0063A201DFEC75A20022E58344F8F583E0A9
:10272A00A363A201F0A363A201DFEE75A20022F95E
:10273A0022C002C004C00612FFF0D006D004D002A4
:01274A00226C
:103DE6004572724C656E210A000A496E49503A00C6
:103DF600205544502054696D654750530A00200AE7
:103E0600444154414752414D3A20002043414E20FF
:103E160054696D654750530A002054726173735399
:103E2600656E644552520A000ACEF8C4EBE8EDFB13
:103E360043414E210A000A45727241647243414E63
:103E46003A00205265496E69742043414E0A0020AB
:103E560043414E283029203E20544F210A00205449
:0C3E66005520300A0020545520310A007D
:03001E00E4FF22DA
:10467F00C2A9438902758C48758A4875D90475DBC0
:10468F004875DC4875DD4875DE48E4F5E9F5F9D283
:08469F00D9C2DAD28CD2DE226E
:1045A800C2D9907B05E07013E5E92419F5EB30D703
:1045B80006E5F904F5FB2285F9FB22E5E924C8F5AF
:0E45C800EB30D706E5F904F5FB2285F9FB225E
:10444200C2D9907B05E0702C302B16E5E92432F5B9
:10445200EB30D707E5F904F5FB800385F9FBC22BA6
:1044620022E5E92405F5EB30D706E5F904F5FB2250
:1044720085F9FB22E5E92432F5EB30D706E5F904AC
:07448200F5FB2285F9FB2286
:1046A70012467F907B05E0C39464500612380B12C4
:1046B70045A8120022D22AE4F556907C1DF0F54554
:0746C700F55AC22BF5582241
:1044CB00EF24FCF545D3940D4010200B077E3D7F68
:1044DB00E6123484E4F545D228229077DD63A201FD
:1044EB00907C0D63A201AF4512263DC228200B0D17
:0E44FB007E3D7FEF7C777DDDAB451231732275
:0F47E800D3EF6480948D5006E55A70028F5A22E9
:101E1B0020D903021EF0202A03021EF0E55A604A65
:101E2B00907468540FFF7D47122634E547640170A8
:101E3B001E907470E0B4FF0ED22C200B127E3D7FEF
:101E4B00F61234848009302C06E4F55A021EF01287
:101E5B0045A812364D200B0D7E3E7F047C747D68A9
:101E6B00AB5A123173E4F55A807BE5456043907CA5
:101E7B0011E02405F527D3940D4007E4F545D2284E
:101E8B008063907C0DE527540FFF7D47122634E5C8
:101E9B004730E702D22BE547B40109302C06E54A5F
:101EAB006401600312364D1245A8E4F545D2288033
:101EBB0034E557601E907AF1540FFF7D471226349C
:101ECB00E547B40103202C0312364D1245A8E4F567
:101EDB0057801220100C907B05E0C39464500312C2
:101EEB00408A1245A8123BA18F27EF7003021FA354
:101EFB00124442E4F558E547547EB5470312434775
:101F0B00E547B4010CD22C200B077E3E7F11123417
:101F1B0084E559C394C8501B30031874062559F532
:101F2B0082E4347BF583E5272559F5597D47AF27A7
:101F3B0012262B300121E54720E71C9079DD7D47E8
:101F4B00AF2712262BAF271239ABEF700A200B07E6
:101F5B007E3E7F1F123484E5475481703BE527D3C7
:101F6B00940D400C200B317E3E7F2E123484802842
:101F7B00E549D39407401C200B1E9075697D47AF34
:101F8B002712262B7E3E7F3C7C757D69AB27123159
:101F9B00738005AF27122F16300E1A300015907B69
:101FAB0005E0C39464500C0558E55894F04004C206
:101FBB00AF80FEC20E2002030220C6906001E00437
:101FCB00F07006906000E004F0E5566031D39401A8
:101FDB00400415568028907C1DE004F0E0D3940358
:101FEB00400D200B077E3E7F481234841246A720FB
:101FFB000B077E3E7F55123484E4F556D22A3029E6
:10200B0043E557703F907AF104F0A37408F0A37482
:10201B0080F0A37401F0A37406F0907C08E0907A32
:10202B00F6F0907C09E0907AF7F0907C0AE0907AD9
:10203B00F8F0907C0BE0907AF9F0E4A3F0A3F07544
:10204B00570BC229302772907C06E07035E557702C
:10205B0031907AF17442F0A37408F0907C07E09011
:10206B007AF3F0907C0CE0907AF4F0A37401F075A5
:10207B005706200B077E3E7F64123484907C06E06B
:10208B0004F0907C06E06402702FE557702B907A79
:10209B00F17402F0A37408F0907C07E0907AF3F0EF
:1020AB00A3F0A37401F0755706200B077E3E7F6BE0
:1020BB00123484907C06E004F0C202122C3EC20063
:0120CB0022F2
:10457500E559602CE49078D9F0A3E559F0907ADEFE
:10458500E09078DBF0A37419F0907B0663A20190AC
:1045950078DD63A201AF5912263DE4F5597F01226A
:0345A5007F002272
:0B481E00302805C2287F01227F002205
:0100210022BC
:06484800E4F559F54522DC
:0A482900E4907569F0A3F0A3F022FB
:0748410020457272210A00FC
:1047B200EF600A7B10E4FD7F0C12462C227B107DF9
:0747C200107F0C12462C22AF
:10380B00D29475C353C29475C5C0E5C4B480FB850F
:10381B00C528D2947DE07F0F12473A907B05E04498
:10382B0080FD7F2A12473A7D247F2912473A7D0477
:10383B007F2812473AE4FD7F2B12473A752A20E482
:10384B00F529E4FDAF2A12473A052A0529E529C3D4
:10385B00940840EEE4F52AF529E4FDAF2A12473A25
:10386B00052A0529E529C3940C40EE7D087F051236
:10387B00473A752A10E4F529E4FDAF2A12473A05B9
:10388B002A0529E529C3940C40EE7D3C7F0C124799
:10389B003A7D077F0F12473A7DFF7F2B12473A7510
:1038AB002A30E4F528E4F529E4FDAF2A12473A055E
:1038BB002A0529E529C3940E40EE052A052A052879
:1038CB00E528C3940340DE7D047F6012473AE4FD94
:0538DB007F7012473A66
:0138E00022C5
:10471600C29475C503E5C4B480FBAEC58FC5E5C4B8
:10472600B480FBAEC5E4F5C5E5C4B480FBAEC5D226
:0347360094AF0637
:01473900225D
:10473A00C29475C502E5C4B480FBAEC58FC5E5C495
:10474A00B480FBAEC58DC5E5C4B480FBAEC5D294BA
:01475A00223C
:10462C00C29475C505E5C4B480FBAEC58FC5E5C4A1
:10463C00B480FBAEC58BC5E5C4B480FBAEC58DC5DF
:09464C00E5C4B480FBAEC5D294B4
:014655002242
:10372D00C29475C503E5C4B480FBAEC5EF60047EDD
:10373D007080027E608EC5E5C4B480FBAEC5E4F535
:10374D00C5E5C4B480FB85C546E4F5C5E5C4B480C4
:10375D00FB85C547E4F5C5E5C4B480FB85C548E4E4
:10376D00F5C5E5C4B480FB85C549E4F5C5E5C4B42C
:10377D0080FB85C54AE4F5C5E5C4B480FB85C54B22
:10378D00E54B540FFE60741EE4F5C5E5C4B480FB33
:10379D0085C54CEE60651EE4F5C5E5C4B480FB85BA
:1037AD00C54DEE60561EE4F5C5E5C4B480FB85C578
:1037BD004EEE60471EE4F5C5E5C4B480FB85C54FEC
:1037CD00EE60381EE4F5C5E5C4B480FB85C550EE4A
:1037DD0060291EE4F5C5E5C4B480FB85C551EE60D6
:1037ED001A1EE4F5C5E5C4B480FB85C552EE600B29
:0D37FD00E4F5C5E5C4B480FB85C553D29446
:01380A00229B
:10364D00907B05E0C39464400302372AC29475C58C
:10365D0002E5C4B480FBAFC575C531E5C4B480FBCC
:10366D00AFC5E54B540FFE8547C5E5C4B480FBAF30
:10367D00C58548C5E5C4B480FBAFC58549C5E5C45E
:10368D00B480FBAFC5854AC5E5C4B480FBAFC58525
:10369D004BC5E5C4B480FBAFC5EE606C1E854CC553
:1036AD00E5C4B480FBAFC5EE605E1E854DC5E5C4B7
:1036BD00B480FBAFC5EE60501E854EC5E5C4B48029
:1036CD00FBAFC5EE60421E854FC5E5C4B480FBAFB0
:1036DD00C5EE60341E8550C5E5C4B480FBAFC5EEA4
:1036ED0060261E8551C5E5C4B480FBAFC5EE6018DC
:1036FD001E8552C5E5C4B480FBAFC5EE600A855387
:10370D00C5E5C4B480FBAFC5D2947F02C29475C524
:0F371D0081E5C4B480FBAFC5D29475560AC22AA9
:01372C00227A
:10434700C29475C502E5C4B480FBAFC575C541E528
:10435700C4B480FBAFC58547C5E5C4B480FBAFC512
:104367008548C5E5C4B480FBAFC58549C5E5C4B478
:1043770080FBAFC5854AC5E5C4B480FBAFC5E4F58E
:10438700C5E5C4B480FBAFC5D2947F02C29475C59E
:0A43970082E5C4B480FBAFC5D294E8
:0143A10022F9
:10408A00C29475C502E5C4B480FBAFC575C551E5D8
:10409A00C4B480FBAFC57472250FF582E43461F5B0
:1040AA0083E0F5C5E5C4B480FBAFC575C508E5C4B2
:1040BA00B480FBAFC57473250FF582E43461F583D0
:1040CA00E0F5C5E5C4B480FBAFC575C50FE5C4B45A
:1040DA0080FBAFC5050F050F7472250FF582E43416
:1040EA0061F583E07002F50FE4F5C5E5C4B480FB21
:1040FA00AFC5D2947F02C29475C584E5C4B480FB6F
:04410A00AFC5D294D7
:01410E00228E
:103BA1003092037F00227F2C1247168F28E52830A0
:103BB100E209D22AE4F556907C1DF0E52830E5585B
:103BC100200B077E487F411234847F2D1247168FC8
:103BD10029200B11E528FE7C00E42529FFEC3EFE9F
:103BE1007D0312356CE4FBAD297F2D12462C200B91
:103BF1001BE52830E016E4FF12372DE547FE7C0077
:103C0100E4254BFFEC3EFE7D0312356CAB28E4FD51
:103C11007F2C12462C7F0022E4F529E52830E00DA7
:103C2100E4FF12372DE54B54072405F529AB28E4B1
:083C3100FD7F2C12462CAF2987
:013C39002268
:10130B005452414E5A004D415842005254530044DE
:10131B00454C4159004E4F4B5654004B5000424FD9
:10132B004F540043414E004E4557504B54004154CF
:10133B00004443440043414E4D4F4E0054454C3AFC
:10134B00004C434C0044544200003E2A2C312CCF1D
:10135B00E0F0E0ECE5F2F0FB20F3EFF0E0E2EBFF86
:10136B00FEF9E5E3EE20EAEEEDF2F0EEEBEBE5F065
:10137B00E020CACF20C8F1E5F2FC0A003E4C2C6BF2
:10138B0030312C25732C43EAEEF0EEF1F2FC20ED1C
:10139B00E020F8E8EDE52043414E2C30202D2035A0
:1013AB003030EAE1283530EC292C31202D20353036
:1013BB00EAE128353030EC290A0030202D20353079
:1013CB0030EAE1283530EC290031202D203530EA88
:1013DB00E128353030EC29003E532C6B30322C2574
:1013EB0062752CCCE0EAF12E20E0E4F0E5F120E18F
:1013FB00EBEEEAE020D2D128302D38290A003E53FB
:10140B002C6B30332C2562752CCCE0EAF12E20E0CE
:10141B00E4F0E5F120E1EBEEEAE020D2C8D228308F
:10142B002D38290A003E532C6B30342C2562752C39
:10143B00CCE0EAF12E20E0E4F0E5F120E1EBEEEA7E
:10144B00E020D2D328302D38290A003E422C6330BD
:10145B00312C2562752CC2F2EEF0E8F7EDFBE9209A
:10146B00EAEEEDF2F0EEEBEBE5F020EDE020F8E844
:10147B00EDE50A003E2A2C312CCFE0F0E0ECE5F252
:10148B00F0FB20EFF0EEF2EEEAEEEBE020C8F1E538
:10149B00F2FC20EFEE20EFEEF0F2F320525332335A
:1014AB00320A003E4C2C6B30352C256C752CD1EA56
:1014BB00EEF0EEF1F2FC20EEE1ECE5EDE020EDE0FC
:1014CB0020EFEEF0F2F32C3130302C3230302C3365
:1014DB0030302C3630302C313230302C32343030FE
:1014EB002C343830302C393630302C3139323030D6
:1014FB002C33383430302C35373630302C313135C5
:10150B003230300A003C21003C6B30313D003C6BEB
:10151B0030323D003C6B30333D003C6B30343D0092
:10152B003C6330313D003C6B30353D0043796354B7
:10153B00530A004D6573730A00435449490A00432B
:10154B005449540A0053705449540A0054696D6548
:10155B005449540A000A4173796E634F55543A004B
:10156B00CEF820E4EBE8EDFB210A000A43524320BE
:10157B004552523A20000A494E3A000A4173796E9D
:10158B0063494E3A003F3F3F0A000089129B24AD4E
:10159B0036BF48C15AD36CE57EF78108931AA52C48
:1015AB00B73EC940DB52ED64FF76028B109926AF34
:1015BB0034BD4AC358D16EE77CF5830A9118A72E28
:1015CB00B53CCB42D950EF66FD74048D169F20A914
:1015DB0032BB4CC55ED768E17AF3850C971EA12808
:1015EB00B33ACD44DF56E960FB72068F149D22ABF4
:1015FB0030B94EC75CD56AE378F1870E951CA32AE8
:10160B00B138CF46DD54EB62F97008811A932CA5E3
:10161B003EB740C952DB64ED76FF89009B12AD24C7
:10162B00BF36C148D35AE56CF77E0A8318912EA7B3
:10163B003CB542CB50D966EF74FD8B029910AF26A7
:10164B00BD34C34AD158E76EF57C0C851E9728A193
:10165B003AB344CD56DF60E972FB8D049F16A92087
:10166B00BB32C54CD75EE168F37A0E871C952AA373
:10167B0038B146CF54DD62EB70F98F069D14AB2267
:10168B00B930C74ED55CE36AF17800112332465767
:10169B0065748C9DAFBECADBE9F810013322564747
:1016AB0075649C8DBFAEDACBF9E8213002136776F7
:1016BB004455ADBC8E9FEBFAC8D931201203776627
:1016CB005445BDAC9E8FFBEAD8C9425361700415DB
:1016DB002736CEDFEDFC8899ABBA52437160140507
:1016EB003726DECFFDEC9889BBAA637240512534B7
:1016FB000617EFFECCDDA9B88A9B736250413524E7
:10170B001607FFEEDCCDB9A89A8B8495A7B6C2D38A
:10171B00E1F008192B3A4E5F6D7C9485B7A6D2C3C6
:10172B00F1E018093B2A5E4F7D6CA5B48697E3F276
:10173B00C0D129380A1B6F7E4C5DB5A49687F3E2A6
:10174B00D0C139281A0B7F6E5C4DC6D7E5F480915A
:10175B00A3B24A5B69780C1D2F3ED6C7F5E4908186
:10176B00B3A25A4B79681C0D3F2EE7F6C4D5A1B036
:10177B0082936B7A48592D3C0E1FF7E6D4C5B1A066
:10178B0092837B6A58493D2C1E0FFF130BFF1311DD
:10179B00FF1316FF131AFF1320FF1326FF1329FF46
:1017AB00132EFF1332FF1339FF133CFF1340FF13AC
:0A17BB0047FF134CFF1350FF1354B7
:0300230002306A3E
:0B306A00C0E0C083C082C0D075D01849
:1030750030984AC298750B01AF9920110DEF640283
:10308500703B90616CF0D2118033301807C2185331
:103095001F0F801ABF0904D2188022BF0310856153
:1030A5006C636180536180C211750B00800F7421C0
:1030B5002561F582E4346FF583EFF005612099030E
:1030C50002316A201203023168301762E568B4FFE5
:1030D5000B7599020568756D00023168E568B56084
:1030E500077599030568807BE568D395604006C23E
:1030F50012D21D806EE56D6009F5990568756D0044
:10310500806174212568F582E43470F583E0F56DFE
:103115006402600BE56D64036005E56DB409057532
:103125009909803F856D990568756D008035742115
:103135002568F582E43470F583E0FF7006C212D28B
:103145001D8020C21DEFB47C090568750832C212C6
:103155008011AF68056874212FF582E43470F5831A
:05316500E0F599C2999C
:09316A00D0D0D082D083D0E03235
:103A5B007BFF7A137955121827907B05E07014754C
:103A6B002FFF7530137531C57BFF7A1379871218C9
:103A7B00278012752FFF7530137531D47BFF7A13A6
:103A8B0079871218277BFF7A1379E3906171E0F540
:103A9B002F1218277BFF7A14790990616BE0F52FB1
:103AAB001218277BFF7A147930906102E0F52F1200
:103ABB0018277BFF7A147956A210E433F52F1218CE
:103ACB00277BFF7A14797F121827907462E0FEA38C
:103ADB00E0FFC3E49FFFE49EFEAB07FAE4F9F8FFB7
:103AEB007E8C7D0AFC1221648F328E318D308C2FAF
:0A3AFB007BFF7A1479AE121827221F
:10327A007E157F10123F80EF4E70037F0122E4908B
:10328A007B05F07E157F13123F80EF4E60151247C3
:10329A0098BF3106907B05740AF0BF3206907B0511
:1032AA007464F07E157F19123F80EF4E6008124257
:1032BA00EA906171EFF07E157F1F123F80EF4E603A
:1032CA00081242EA90616BEFF07E157F25123F806B
:1032DA00EF4E60081242EA906102EFF07E157F2BF2
:1032EA00123F80EF4E600D1242EAEC4D4E4F24FF22
:1032FA0092108002C2107E157F31123F80EF4E601D
:10330A000D1242EA8F2A8E298D288C27800A907402
:10331A00627425F0A37480F0AB2AAA29A928A827E9
:10332A007F007E8C7D0A7C001221641221F6907443
:10333A0062EEF0A3EFF0E47F587E02FDFCAB2AAA0E
:10334A0029A928A827D31222045007756901D2197E
:10335A008021E47F607E09FDFCAB2AAA29A928A85E
:10336A0027D31222045007756902C21980057569AC
:05337A0004C2197F00F0
:01337F00222B
:10274B00E4F50F907C31F0907C31E075F003A4241C
:10275B0095F582E43417F583E493FB740193FA74D3
:10276B000293F91220CC7003022912E4907C33F00F
:10277B00A3F0907C32F0907C32E02491F582E4342B
:10278B0075F583E0FF7003022909907C31E075F049
:10279B0003A42495F582E43417F583E493FB7401C9
:1027AB0093FA740293F9907C33E0F58275830012EF
:1027BB0020E5FEEFB5060F907C347401F0907C336E
:1027CB00E004F0022900907C34E07003022900EE53
:1027DB0060030228F7907C31E014606E24FC7003D8
:1027EB000228C11470030228EF14700302289124ED
:1027FB00F970030228F3240E6003022909907C323E
:10280B00E02491F9E43475FA7B01C0031B8B2E7520
:10281B002F00753000E4F531D003122913907C356D
:10282B00122215907C35E0F8A3E0F9A3E0FAA3E0BF
:10283B00FB7F007E8C7D0A7C001221641221F690B6
:10284B007462EEF0A3EFF0022909907C32E0FD24D4
:10285B0091F582E43475F583E024D0906171F074C6
:10286B00922DF582E43475F583E024D090616BF002
:10287B00907C32E02493F582E43475F583E024D028
:10288B00906102F08078907C32E02491F9E4347509
:10289B00FA7B01C0031B8B2E752F00753000E4F5FE
:1028AB0031D003122913907C35122215907C38E01D
:1028BB00907B05F08048907C32E02491F9E43475EC
:1028CB00FA7B01C0031B8B2E752F00753000E4F5CE
:1028DB0031D003122913907C35122215907C38E0ED
:1028EB00F56B801AD2138016D2198012E4907C34C7
:1028FB00F0907C33F0907C32E004F0022781907CE6
:07290B0031E004F002275245
:0129120022A2
:10235F00E4906170F09061B5F0C21690616EF090EC
:10236F006F1E7405F0C212C21DC211C218E4F568C7
:10237F00F560F508F561F50B90746274FFF0A374C6
:10238F00F4F09061027402F090616BF0906171F063
:10239F00C21BD21AC210907121741EF0E4907B05FB
:1023AF00F0C213C215C214F56BC219D21712327ACA
:1023BF00EF600312274B907121E00490616DF0E400
:1023CF00F50F907C2F7461F0A37472F0906171E03F
:1023DF00F50FE50FC394014007E50FD394084003B1
:1023EF00E4F50FE50F6028907C2FE475F0011221C2
:1023FF001285F082F58374C4F0150F907C2FE4756D
:10240F00F00112211285F082F583E50FF080D49050
:10241F00616BE0F50FE50FC394014007E50FD3940F
:10242F00084003E4F50FE50F6028907C2FE475F06A
:10243F000112211285F082F58374C8F0150F907C7C
:10244F002FE475F00112211285F082F583E50FF06C
:10245F0080D4906102E0F50FE50FC394014007E5CA
:10246F000FD394084003E4F50FE50F6028907C2FFD
:10247F00E475F00112211285F082F58374C2F01514
:10248F000F907C2FE475F00112211285F082F583F5
:10249F00E50FF080D4907C2FE475F00112211285A6
:1024AF00F082F583E4F0907C2F75F00112211285F4
:1024BF00F082F583E4F0F50FF56A75F075E56AA41F
:1024CF002436F582E5F03468F583E4F0E56A75F0BB
:1024DF000DA42403F582E43461F583E4F0F55F7510
:1024EF00F068E56AA42422F582E5F03471F583756E
:1024FF00F00DE55F122252E4F0055FE55FB408DFEF
:10250F00056AE56AB408B3E4F56FF55BF55DF55E52
:10251F00F567F56EF55FF55CF56AF566F59BC2AD8F
:10252F00F5C9D2CDD2CCC2C9C2CAF5CDF5CC907403
:10253F0062E0F5CBA3E0F5CA85CBCD85CACCD29EA0
:10254F00D29CD2CAC2ACC298C29975B81075B710D6
:02255F00D2ACFC
:012561002257
:0100220022BB
:102F16008F2830190EE547B44209E54A640270036A
:102F2600023069E54854E324DF606D24DF60421413
:102F3600603F24E37003022FC51470030230171498
:102F4600700302304824E26028246060030230697E
:102F5600300C077E157F37123484E54975F00DA4D1
:102F66002403F582E43461F5837D47AF2812262BCE
:102F760022300C077E157F3E12348475F00DE55E17
:102F8600A424DEF582E5F0346BF5837D47AF281285
:102F9600262B055E535E3F22300C077E157F4412BA
:102FA600348475F00DE55BA424B6F582E5F0346152
:102FB600F5837D47AF2812262B055B535B7F2230B6
:102FC6000C077E157F4A12348475F075E549A424F2
:102FD60043F582E5F03468F583E54A541FFF131381
:102FE600543F75F00D1222527D47AF2812262B75DD
:102FF600F068E549A42422F582E5F03471F583E50D
:103006004A541FFF1313543F75F00D122252E4F079
:1030160022300C077E157F5012348475F068E5491E
:10302600A42422F582E5F03471F583E54A543FFF86
:103036001313543F75F00D1222527D477F0D122651
:103046002B22300C077E157F5712348475F075E5F8
:1030560049A42436F582E5F03468F5837D47AF2828
:0430660012262B22E1
:103CCA008F2B90600263A20190702163A201AF2B37
:103CDA0012263DE4F562F563852B6590702163A297
:103CEA000190159563A201AF65AE64AD63AC621233
:103CFA0026798F658E648D638C627421252BF582FB
:103D0A00E43470F583E563F07422252BF582E434FC
:103D1A0070F583E562F07421252BF582E43470F5A1
:103D2A0083E0FFA3E0906F1FCFF0A3EFF0E52B2411
:103D3A0002F5607F011247B27568FFD212D299204C
:103D4A000B0D7E157F607C707D21AB601231732272
:101B2100E55E655D605875F00DE55DA424E2F58222
:101B3100E5F0346BF583E02405F52BD3940E400CCE
:101B4100200B357E157F6B123484802C75F00DE5EA
:101B51005DA424DEF582E5F0346BF58363A20174A4
:101B6100042566F582E43460F58363A201AF2B128C
:101B7100263DE52B2566F566055D535D3F2275F033
:101B810075E56AA42436F582E5F03468F583E070E2
:101B910003021C88E55C705575F075E56AA4243A6A
:101BA100F582E5F03468F583E02405F52BD3940E36
:101BB100400C200B357E157F6B123484802C75F020
:101BC10075E56AA42436F582E5F03468F58363A2ED
:101BD1000174042566F582E43460F58363A201AFE4
:101BE1002B12263DE52B2566F566055C2275F07501
:101BF100E56AA42439F582E5F03468F583E0540FF1
:101C0100FFE55CD39F506575F075E56AA4243AF54C
:101C110082E5F03468F58375F00DE55C122252E03F
:101C21002405F52BD3940E400C200B3D7E157F6BC4
:101C3100123484803475F075E56AA42436F582E5A2
:101C4100F03468F58375F00DE55C12225263A20150
:101C510074042566F582E43460F58363A201AF2B39
:101C610012263DE52B2566F566055C22E4F55C75DB
:101C7100F075E56AA42436F582E5F03468F583E46D
:101C8100F0056A536A0722056A536A07E55B656FC7
:101C9100605875F00DE56FA424BAF582E5F0346162
:101CA100F583E02405F52BD3940E400C200B357EF3
:101CB100157F6B123484802C75F00DE56FA424B66A
:101CC100F582E5F03461F58363A20174042566F5BC
:101CD10082E43460F58363A201AF2B12263DE52B2C
:101CE1002566F566056F536F7F22E56775F00DA4D4
:101CF1002403F582E43461F583E06067E56775F0FC
:101D01000DA42407F582E43461F583E02405F52B65
:101D1100D3940E400C200B347E157F6B12348480DB
:101D21002BE56775F00DA42403F582E43461F58396
:101D310063A20174042566F582E43460F58363A22D
:101D410001AF2B12263DE52B2566F566E56775F09B
:101D51000DA42403F582E43461F583E4F0056753AF
:101D6100670722056753670775F068E56EA42422AB
:101D7100F582E5F03471F58375F00DE55F122252BD
:101D8100E07003021E0975F068E56EA42426F58251
:101D9100E5F03471F58375F00DE55F122252E02410
:101DA10005F52BD3940E400C200B3D7E157F6B1255
:101DB1003484803475F068E56EA42422F582E5F060
:101DC1003471F58375F00DE55F12225263A201743F
:101DD100042566F582E43460F58363A201AF2B121A
:101DE100263DE52B2566F56675F068E56EA424228F
:101DF100F582E5F03471F58375F00DE55F1222523D
:101E0100E4F0055F535F0722055FE55FC394084077
:091E110008E4F55F056E536E074D
:011E1A0022A5
:102C3E00300010C20090616FE004F09061B5E0606A
:102C4E000214F0E508B40107E4F508D212D299E5B2
:102C5E000BD394644007C211E4F561F50B30120FEB
:102C6E0090616FE0D39414400BC212D21D8005E424
:102C7E0090616FF020123EE508703A301A37F52851
:102C8E00E528C395695010121B21E5666009D3949F
:102C9E00C85004052880E9E566601AE4906002F0E9
:102CAE00A37419F0E5662402FF123CCAE4F566909F
:102CBE006000F0A3F0E56C7003022DAFF528E4F58B
:102CCE006CF562F563E528547FF565E5285480249C
:102CDE0021F582E4346FF58363A20190159563A20A
:102CEE0001AF65AE64AD63AC621226798F658E64FA
:102CFE008D638C62E52854802421F582E4346FAF15
:102D0E0082F5298F2A53287FE5634562601D300BBB
:102D1E0003022DAF7E157F76AB28AD2AAC2912317A
:102D2E00737D03AF63AE6212356C22200B2490616B
:102D3E0070E06401600F7E157F81AB28AD2AAC294F
:102D4E00123173800D7E157F86AB28AD2AAC291209
:102D5E003173E528B40408E490616DF0C21C22853D
:102D6E002A82852983A3E024E7702CD216E5282435
:102D7E00FCF557C3940E501BE52A2402FFE43529B7
:102D8E00F5838F8263A201907AF163A201AF57128D
:102D9E00263D22E4F55722200B077E157F90123434
:012DAE0084A0
:012DAF002201
:103D6600020881E493A3F8E493A34003F68001F2EA
:103D760008DFF48029E493A3F85407240CC8C3335E
:103D8600C4540F4420C8834004F456800146F6DF2D
:103D9600E4800B0102040810204080904833E47E42
:103DA600019360BCA3FF543F30E509541FFEE49322
:103DB600A360010ECF54C025E060A840B8E493A3E9
:103DC600FAE493A3F8E493A3C8C582C8CAC583CA14
:103DD600F0A3C8C582C8CAC583CADFE9DEE780BECC
:01483900007E
:1020CC00BB010689828A83E0225002E722BBFE0212
:0920DC00E32289828A83E4932245
:1020E500BB010CE58229F582E5833AF583E02250B0
:1020F50006E92582F8E622BBFE06E92582F8E222FA
:0D210500E58229F582E5833AF583E4932213
:10211200A3F8E0C5F025F0F0E58215827002158380
:06212200E0C838F0E822DD
:1021280075F008758200EF2FFFEE33FECD33CDCC6E
:1021380033CCC58233C5829BED9AEC99E5829840F1
:102148000CF582EE9BFEED9AFDEC99FC0FD5F0D6CE
:10215800E4CEFBE4CDFAE4CCF9A88222B800C1B9F8
:102168000059BA002DEC8BF084CFCECDFCE5F0CB36
:10217800F97818EF2FFFEE33FEED33FDEC33FCEB6F
:1021880033FB10D703994004EB99FB0FD8E5E4F92A
:10219800FA227818EF2FFFEE33FEED33FDEC33FC17
:1021A800C933C910D7059BE99A4007EC9BFCE99A0B
:1021B800F90FD8E0E4C9FAE4CCFB2275F010EF2F50
:1021C800FFEE33FEED33FDCC33CCC833C810D70750
:1021D8009BEC9AE899400AED9BFDEC9AFCE899F88B
:0E21E8000FD5F0DAE4CDFBE4CCFAE4C8F9221E
:0E21F600C3E49FFFE49EFEE49DFDE49CFC22FA
:10220400EB9FF5F0EA9E42F0E99D42F0E89C45F030
:0122140022A7
:0C221500ECF0A3EDF0A3EEF0A3EFF0223C
:10222100A8828583F0D083D08212223812223812FC
:102231002238122238E473E493A3C583C5F0C58321
:10224100C8C582C8F0A3C583C5F0C583C8C582C807
:01225100226A
:0C225200A42582F582E5F03583F5832297
:1017C500E53B242FF8E6053B22782C302502782FBF
:1017D500E475F0011222BF0220CC201EEB7F2ED231
:1017E5001E8018EF540F2490D43440D4FF30220BC0
:1017F500EF24BFB41A0050032461FFE53C600215D5
:101805003C053FE53F7002053E30250D782CE4751B
:10181500F0011222BFEF02225E0243FB7403D225C0
:101825008003E4C225F53B8B2C8A2D892EE4F53CFB
:10183500F53EF53FE53C60077F2012180080F57501
:101845003DFFC21FC21EC220C221C223C224C2261E
:101855001217CEFF700D3025057F00121811AF3F0E
:10186500AE3E22B4255FC2D5C2221217CEFF24D0C8
:10187500B40A00501A75F00A783C30D50508B6FF51
:101885000106C6A426F620D5047002D22180D924EB
:10189500CFB41A00EF5004C2E5D222021A11D21FAA
:1018A50080C6D21E80C0D22080BCD2D580BAD223B9
:1018B50080B47F201218002020077401B53C004039
:1018C500F11217C5FF121800021839D226D224804A
:1018D500951217C5FB1217C5FA1217C5F94A4B70B1
:1018E5000679E27A1A7BFF20202EE53C602A7E00ED
:1018F5008E827583001220E560060EEE653D70F060
:10190500C2D5EBC0E0EAC0E0E9C0E0EE121A58D05B
:10191500E0F9D0E0FAD0E0FB1220CCFF60AAEBC0E2
:10192500E0EAC0E0E9C0E0121800D0E02401F9D0F7
:10193500E03400FAD0E0FBE53D0460DCD53DD9801C
:10194500877BFF7A1A7954D220809C79108002799E
:1019550008C224C2268008D2D5790A8004790AC231
:10196500D5E53D047002F53DE4FAFDFEFF1217C50D
:10197500FC7B08201F131217C5FD7B10301E0A12B1
:1019850017C5FE1217C5FF7B20EC3382D592D550C3
:1019950013C3E4301E069FFFE49EFEE4201F039D53
:1019A500FDE49CFCE4CBF8C21FEC700CCFCECDCC93
:1019B500E824F8F870F38017C3EF33FFEE33FEED3C
:1019C50033FDEC33FCEB33FB994002FB0FD8E9EB1D
:1019D500301F05F8D0E0C448B21FC0E00AEC4D4EF8
:1019E5004F78207B0070C2EAB53D0040BCC0E012D4
:1019F5001A5AD0F0D0E0201F04C4C0E0C4B21FC002
:101A0500F01217E9D0F0D5F0EB02183912231E18A1
:101A1500D65319505818A74C18A34219544F195C9E
:0F1A250044195C4918BC431962551946461946C5
:101A3400451946471B025018AB2D18AF2E18D22B50
:101A440018B32318D0201AEB2A186B48000018CAC0
:101A54003F3F3F00790AA2D5202114302309B91051
:101A6400020404B9080104A2D52024025001042070
:101A740020689220B53C005034C0E07F203021190A
:101A84007F30A22072247223500F121AB1C220C2D6
:101A940024C223C2267F30800F302303E9C0E01222
:101AA4001800302303D0E0F9D0E0B53CCC30231744
:101AB4007F30B9100C1218007F583022077F7880CD
:101AC40003B908031218003020057F2D0218007F87
:101AD400202026F87F2B2024F322922080CF286E0A
:101AE400756C6C2900D21F1217C5301FF8C21F78FD
:101AF4003C30D50108F602186B2D50434958121793
:101B0400C52403B405004001E4901AFD931217F1B3
:0D1B1400743A1217F1D221753C04021950E9
:102913008B2B8A2C892DE4F537F536F535F534F50F
:1029230032F533E52F4530452E6012EBC0E0EAC0A7
:10293300E0E9C0E0AB2EAA2FA9301222CFAB2B05C2
:102943002DE52DAA2C7002052C14F91220CCF53894
:10295300C394094007E538D3940D40E1E53864207A
:1029630060DBE538B42D054333038016E538B42B1B
:1029730005433301800C74FF252DF52D74FF352C91
:10298300F52CE53160046410703FAB2BAA2CA92D04
:102993001220CC64306009E531702E75310A80292C
:1029A3009000011220E5FF64786004EFB4581343EC
:1029B30033017531107402252DF52DE4352CF52CDA
:1029C3008007E5317003753108AB2B052DE52DAA82
:1029D3002C7002052C14F91220CCF538C3946140F5
:1029E3000AE538D3947A50035338DF74D02538F589
:1029F30038C3940A400CE5389411406D74F92538B6
:102A0300F538E538D39531506043330185373C853C
:102A1300363B85353A853439AF317E00E4FCFDAB76
:102A230037AA36A935A834122270C8ECC8C9EDC933
:102A3300CAEECACBEFCBE4FCFDFEEB2538F537EE4F
:102A43003AF536ED39F535EC38F534AF37AE36AD0A
:102A530035FCAB3CAA3BA93AA839D3122204500354
:102A63000229CC4333040229CCE53320E003E4807C
:102A73002DE52F4530452E601EAB2BE52D24FFF9A8
:102A8300E52C34FFFAEBC0E0EAC0E0E9C0E0AB2E8E
:102A9300AA2FA9301222CFE53330E20774FFFFFEDD
:102AA300FDFC22E533AF37AE36AD35AC3430E10350
:042AB3000221F622E4
:10225E00BB010689828A83F0225002F722BBFE015F
:02226E00F32259
:10227000E88FF0A4CC8BF0A42CFCE98EF0A42CFC0D
:102280008AF0EDA42CFCEA8EF0A4CDA8F08BF0A48B
:102290002DCC3825F0FDE98FF0A42CCD35F0FCEBEA
:1022A0008EF0A4FEA9F0EB8FF0A4CFC5F02ECD39AF
:0F22B000FEE43CFCEAA42DCE35F0FDE43CFC221C
:1022BF00FAE6FB0808E6F925F0F618E6CA3AF62220
:1022CF00BB011A89828A83D0F0D0E0F8D0E0F9D030
:1022DF00E0FAD0E0FBE8C0E0C0F002234D5016E971
:1022EF00F8D083D082D0E0F9D0E0FAD0E0FBC08202
:1022FF00C083022344BBFE16E9F8D083D082D0E01E
:0F230F00F9D0E0FAD0E0FBC082C083022356224F
:10231E00D083D082F8E4937012740193700DA3A34E
:10232E0093F8740193F5828883E473740293686062
:06233E00EFA3A3A380DF62
:09234400EBF608EAF608E9F622BE
:09234D00EBF0A3EAF0A3E9F02291
:09235600EBF208EAF208E9F222B8
:00000001FF
